:0200000480007A
:10000000B72F0000938F0F8073900F3015A8130047
:100010000000130000001300000013000000130094
:100020000000130000001300000013000000130084
:100030000000130000001300000013000000010086
:10004000970200009382020C73905230814001416C
:100050008141014281420143814301448144014580
:100060008145014681460147814701488148014950
:100070008149014A814A014B814B014C814C014D20
:10008000814D014E814E014F814F971102009381A6
:1000900021B7170502001305E53A979503009385EC
:1000A000256801461122170502001305A53497059E
:1000B00002009385A5340146C52817A50300130542
:1000C000656697B503009385A56537B6ABAB130698
:1000D000B6BAD92817B103001301C164EF40D01E8E
:1000E000860293D21200F512638802008242110147
:1000F0006F00001073002030824211017300203025
:10010000711116C0F3222034E3CC02FC82421101AB
:10011000130141F806C20AC40EC612C816CA1ACC88
:100120001ECE22D026D22AD42ED632D836DA3ADCC7
:100130003EDEC2C0C6C2CAC4CEC6D2C8D6CADACC97
:10014000DECEE2D0E6D2EAD4EED6F2D8F6DAFADCA7
:10015000FEDE73252034F32510340A8601A07310C7
:10016000153492402241B2414242D2426243F243AC
:10017000025492542255B2554256D2566257F25703
:10018000064896482649B649464AD64A664BF64B33
:10019000065C965C265DB65D465ED65E665FF65F83
:1001A0001301C1077300203010C16374B50011053D
:1001B000E5BF828000000000000000000000000099
:1001C000000000000000000000000000000000002F
:1001D000000000000000000000000000000000001F
:1001E000000000000000000000000000000000000F
:1001F000197106C00AC20EC412C616C81ACA1ECC8D
:1002000022CE26D02AD22ED432D636D83ADA3EDCC6
:1002100042DEC6C0CAC2CEC4D2C6D6C8DACADECC96
:10022000E2CEE6D0EAD2EED4F2D6F6D8FADAFEDCA6
:100230009702020083A2021C23A02200F3221034A2
:1002400096DEEF006030170102000321A11A02417F
:10025000F65273901234B72200009382028873A082
:10026000023082403242C2425243E24372448254DC
:100270001255A2553256C2565257E2577258864806
:100280001649A649364AC64A564BE64B764C865C1A
:10029000165DA65D365EC65E565FE65F0961730059
:1002A0002030970202009382E21923A0120023A2B9
:1002B000220023A4320023A6420023A8520023AA2E
:1002C000620023AC720023AE820023A0920223A21C
:1002D000A20223A4B20223A6C20223A8D20223AA06
:1002E000E20223ACF20223AE020323A0120523A2F2
:1002F000220523A4320523A6420523A8520523AADA
:10030000620523AC720523AE820523A0920723A2C7
:10031000A20723A4B20723A6C20723A8D20723AAB1
:10032000E20723ACF207EF40E06E17010200032161
:10033000610C0241F65273901234B722000093828E
:10034000028873A0023082403242C2425243E243EA
:10035000724482541255A2553256C2565257E25731
:10036000725886481649A649364AC64A564BE64B45
:10037000764C865C165DA65D365EC65E565FE65FB1
:10038000096173002030970202009382A20B83A0C0
:10039000020003A1420083A1820003A2C20083A243
:1003A000020103A3420183A3820103A4C20183A427
:1003B000020203A5420283A5820203A6C20283A60B
:1003C000020303A7420383A7820303A8C20383A8EF
:1003D000020403A9420483A9820403AAC20483AAD3
:1003E000020503AB420583AB820503ACC20583ACB7
:1003F000020603AD420683AD820603AEC20683AE9B
:10040000020703AFC20983AF820782807370043092
:10041000197106C00AC20EC412C616C81ACA1ECC6A
:1004200022CE26D02AD22ED432D636D83ADA3EDCA4
:1004300042DEC6C0CAC2CEC4D2C6D6C8DACADECC74
:10044000E2CEE6D0EAD2EED4F2D6F6D8FADAFEDC84
:100450009702020083A202FA23A0220086DEEF1098
:100460003062170102000321E1F80241F652739055
:100470001234B72200009382028873A002308240B7
:100480003242C2425243E243724482541255A25550
:100490003256C2565257E257725886481649A649F4
:1004A000364AC64A564BE64B764C865C165DA65DD0
:1004B000365EC65E565FE65F0961730020309707BF
:1004C00002009387E7F39843FD576305F7007370C5
:1004D000043001A07370043001A041112AC6B24754
:1004E000739047300100410182804111F327403071
:1004F0003EC673F04330B2473E85410182804111D0
:100500002AC62EC432C2B247F1173EC62247B247AE
:1005100098C3B247938787FA3EC61247B24798C33B
:10052000B247A1173EC68E873E87B24798C3B247EF
:10053000D1173EC6170700001307A7F8B24798C3A4
:10054000B2473E8541018280411106C6EF402045F9
:10055000EF105036AA8799C3EF1090520100B240B5
:100560004101828041112AC6B24713878700B247F2
:10057000D8C3B2477D5798C7B24713878700B247A1
:10058000D8C7B24713878700B24798CBB24723A09A
:10059000070001004101828041112AC6B24723A809
:1005A000070001004101828001112AC62EC4B24712
:1005B000DC433ECEA2477247D8C3F2479847A247D2
:1005C00098C7F2479C472247D8C3F247224798C7AB
:1005D000A247324798CBB2479C4313871700B247D4
:1005E00098C301000561828001112AC62EC4A2476A
:1005F0009C433ECC6247FD576316F700B2479C4BC5
:100600003ECE31A8B247A1073ECE21A0F247DC433F
:100610003ECEF247DC439C436247E379F7FEF24764
:10062000D843A247D8C3A247DC43224798C7A24772
:10063000724798C7F2472247D8C3A247324798CBA0
:10064000B2479C4313871700B24798C30100056166
:10065000828001112AC6B2479C4B3ECEB247DC4392
:100660003247184798C7B2479C4732475843D8C3C8
:10067000F247DC4332476316F700B2479847F24728
:10068000D8C3B24723A80700F2479C431387F7FF5C
:10069000F24798C3F2479C433E8505618280797199
:1006A00006D622D42AC62EC4B2473ECEF24781E7F0
:1006B0007370043001A0EF20A078F2478043F24726
:1006C000D85FF247BC43BE853A85EF50A038AA8771
:1006D0003307F400F247D8C3F24723AC0702F247CE
:1006E0009843F24798C7F2478043F247DC5F13878D
:1006F000F7FFF247BC43BE853A85EF50A035AA8785
:100700003307F400F247D8C7F2477D57F8C3F247E2
:100710007D57B8C7A24799EFF2479C4B8DC7F24768
:10072000C1073E85EF1010622A878547631DF700D9
:10073000F13911A8F247C1073E852D35F24793875D
:1007400047023E850535EF20807285473E85B250D1
:10075000225445618280797106D62AC62EC4B2879A
:10076000A303F10002CCB24781E77370043001A00B
:10077000A24799E302CE01A8A2453245EF50802D51
:10078000AA8785073ECEF247938747053E85EF301F
:10079000007E2ACAD24785CFA24789E7D24752476F
:1007A00098C331A0D24713874705D24798C3D24791
:1007B0003247D8DFD2472247B8C385455245C535B1
:1007C000D247034771002388E704D2473ECCE24773
:1007D00081E77370043001A0E2473E85B250456165
:1007E0008280797106D6AA87A307F1001305400518
:1007F000EF30E0772ACEF247B9CFF24723A20700C5
:10080000F24723A00700F24723A40700F24723A6DC
:100810000700F24723AC0702F2470547D8DFF2474B
:1008200023A00704F2477D57F8C3F2477D57B8C7A6
:10083000F2470347F1002388E704F247C1073E85EA
:100840001533F247938747023E85293B814601468F
:10085000814572453122F2473E85B2504561828022
:10086000797106D622D42AC6B2473ECCE24781E748
:100870007370043001A0E247C043EF20803EAA8796
:100880006313F402E247DC471387F7FFE247D8C758
:10089000E247DC4791E78146014681456245C92030
:1008A00085473ECE11A002CEF2473E85B25022547B
:1008B00045618280797106D622D42AC62EC4B247F9
:1008C0003ECCE24781E77370043001A0E247C043A9
:1008D000EF202039AA87631BF400E247DC47138727
:1008E0001700E247D8C785473ECE0DA08146224675
:1008F00081456245812B2ACE724785476318F700F0
:10090000E247DC4713871700E247D8C7F2473E8526
:10091000B250225445618280797106D62AC62EC40F
:10092000B24781E77370043001A02247B24763F5F4
:10093000E7007370043001A0094681453245213D2E
:100940002ACEF24781C7F247224798DFF24781E774
:100950007370043001A0F2473E85B2504561828039
:10096000397106DE2AC62EC432C236C002D6B2475C
:100970003ED4A25781E77370043001A0A24781E7FB
:10098000A257BC4399E3854711A0814781E7737063
:10099000043001A0024789476317F700A257D85FC8
:1009A00085476314F700854711A0814781E773707D
:1009B000043001A0EF20402CAA8799E3924799E3E5
:1009C000854711A0814781E77370043001A0EF20B3
:1009D0002047A257985FA257DC5F6366F700024783
:1009E0008947631EF7020246A2452255EF00007CAC
:1009F0002AD2A257DC5389CFA257938747023E855C
:100A0000EF1050342A8785476317F700013421A07F
:100A1000925791C3E53AEF20804585474DA0924714
:100A200089E7EF20C044814759A8B25799E77C086D
:100A30003E85EF10D04885473ED6EF204043EF106B
:100A4000A03BEF20E03FA257F843FD576315F700A6
:100A5000A25723A20704A257B847FD576315F70012
:100A6000A25723A40704EF20804058007C08BA85D1
:100A70003E85EF10D047AA878DEF2255EF00D012A8
:100A8000AA8795C3A257C1071247BA853E85EF10C2
:100A900050122255EF00B003EF10C037AA87E39839
:100AA00007F2AD322DB72255EF007002EF108036FD
:100AB00039BF2255EF00B001EF10C03581473E85A8
:100AC000F25021618280797106D62AC62EC432C2C4
:100AD00036C002CEB2473ECCE24781E773700430A5
:100AE00001A0A24781E7E247BC4399E3854711A0F3
:100AF000814781E77370043001A0EF206034E24742
:100B0000985FE247DC5F6379F7020246A2456245DF
:100B1000EF00C069E247DC5381CFE2479387470289
:100B20003E85EF1030222A8785476313F700F93896
:100B3000EF20E033854785A0924789E7EF202033F7
:100B4000814791A8F24799E71C083E85EF1030379E
:100B500085473ECEEF20A031EF20802E58001C08A4
:100B6000BA853E85EF10B038AA8799EF6245EF004D
:100B7000B003AA8791CFE247C1071247BA853E85E5
:100B8000EF103003613029A0EF20602E814721A0B3
:100B9000EF20E02D9DB73E85B250456182803971CE
:100BA00006DE2AC62EC432C236C002D6B2473ED4B2
:100BB000A25781E77370043001A0A24781E7A257D2
:100BC000BC4399E3854711A0814781E773700430E6
:100BD00001A0EF20E026A2579C5FB5CBA257DC47CF
:100BE0003ED2A2452255792D824795EFA2579C5FB0
:100BF0001387F7FFA25798DFA2579C4391E7EF2096
:100C0000602E2A87A257D8C3A2579C4B8DCFA257DC
:100C1000C1073E85EF1010132A8785476315F70239
:100C2000EFF0CFFE0DA0A2571257D8C7A257DC5342
:100C300099CBA257938747023E85EF10B010AA8741
:100C400099C3EFF0AFFCEF2080228547ADA8924713
:100C500089E7EF20C0218147BDA0B25799E77C0802
:100C60003E85EF10D02585473ED6EF204020EF206F
:100C7000201D58007C08BA853E85EF105027AA87B2
:100C800085EF2255E92DAA8785CFA2579C4391EB8A
:100C9000EF20001BA257DC433E85EF20E000EF2051
:100CA000001DA257938747021247BA853E85EF1071
:100CB0004070EFF0AFF529A0EF20601B814721A025
:100CC000EF20E01A39B73E85F250216182807971B8
:100CD00006D62AC62EC432C236C0B2473ECCE24740
:100CE00081E77370043001A0A24781E7E247BC436B
:100CF00099E3854711A0814781E77370043001A013
:100D0000024789476317F700E247D85F85476314B6
:100D1000F700854711A0814781E77370043001A077
:100D2000EFF0AFFCAA873ECAE247985FE247DC5F7C
:100D30006366F700024789476315F7040246A24538
:100D40006245AD21E247B847FD576313F702E2471A
:100D5000DC538DC7E247938747023E85EF10807EC4
:100D6000AA8789CF924799CB9247054798C339A064
:100D7000E247BC4713871700E247B8C785473ECE16
:100D800011A002CED2473E85EFF02FF5F2473E8507
:100D9000B25045618280797106D62AC62EC4B24708
:100DA0003ECCE24781E77370043001A0E247BC43C8
:100DB00081C77370043001A0E2479C4381E7E2479A
:100DC000DC4399E3854711A0814781E773700430C4
:100DD00001A0EFF08FF1AA873ECAE247985FE24791
:100DE000DC5F6377F704E2479C5F13871700E247F5
:100DF00098DFE247B847FD576313F702E247DC5339
:100E00008DC7E247938747023E85EF10A073AA87FC
:100E100089CFA24799CBA247054798C339A0E2479B
:100E2000BC4713871700E247B8C785473ECE11A0DD
:100E300002CED2473E85EFF04FEAF2473E85B250F0
:100E400045618280397106DE2AC62EC432C236C0A0
:100E500002D6B2473ED4A25781E77370043001A096
:100E6000A24781E7A257BC4399E3854711A0814778
:100E700081E77370043001A0EF101060AA8799E336
:100E8000924799E3854711A0814781E77370043049
:100E900001A0EF10F07AA2579C5FB5CBA257DC47B8
:100EA0003ED2A2452255F92E824795EFA2579C5F6C
:100EB0001387F7FFA25798DFA2579C4391E7EF20D3
:100EC00060022A87A257D8C3A2579C4B8DCFA25746
:100ED000C1073E85EF1000672A8785476315F70233
:100EE000EFF0CFD20DA0A2571257D8C7A257DC53AC
:100EF00099CBA257938747023E85EF10A064AA873B
:100F000099C3EFF0AFD0EF10907685475DA8924778
:100F100089E7EF10D07581476DA0B25799E77C083B
:100F20003E85EF10C07985473ED6EF105074EF0034
:100F3000B06CEF10F070A257F843FD576315F7003F
:100F4000A25723A20704A257B847FD576315F7001D
:100F5000A25723A40704EF10907158007C08BA85AB
:100F60003E85EF10C078AA87A1EB2255CD2EAA8727
:100F70009DCFA2579C4391EBEF10906CA257DC439E
:100F80003E85EF107052EF10906EA2579387470284
:100F90001247BA853E85EF10C04122550D2EEF0055
:100FA0007067AA87E39707EEEFF04FC6DDB52255CD
:100FB000392EEF003066F1BD2255112EEF009065FD
:100FC00081473E85F25021618280797106D62AC61A
:100FD0002EC432C2B2473ECCE24781E77370043080
:100FE00001A0A24781E7E247BC4399E3854711A0EE
:100FF000814781E77370043001A0EFF00FCFAA871B
:101000003ECAE2479C5FA1CBA2456245A52CE247C0
:101010009C5F1387F7FFE24798DFE247F843FD57ED
:101020006312F702E2479C4B85C7E247C1073E8542
:10103000EF104051AA8789CF924799CB9247054735
:1010400098C339A0E247FC4313871700E247F8C36F
:1010500085473ECE11A002CED2473E85EFF0EFC7C6
:10106000F2473E85B25045618280797106D62AC624
:101070002EC4B2473ECCE24781E77370043001A032
:10108000A24781E7E247BC4399E3854711A0814726
:1010900081E77370043001A0E247BC4381E77370BD
:1010A000043001A0EFF06FC4AA873ECAE2479C5FFC
:1010B00089CFE247DC473EC8A2456245E122E247CC
:1010C0004247D8C785473ECE11A002CED2473E85C3
:1010D000EFF0AFC0F2473E85B25045618280797132
:1010E00006D62AC6B24781E77370043001A0EF101C
:1010F0003055B2479C5F3ECEEF107057F2473E85A9
:10110000B25045618280797106D62AC6B2473ECE7A
:10111000F24781E77370043001A0EF107052F2477C
:10112000D85FF2479C5FB307F7403ECCEF103054D6
:10113000E2473E85B2504561828001112AC6B2471E
:1011400081E77370043001A0B2479C5F3ECEF24746
:101150003E8505618280797106D62AC6B2473ECEA9
:10116000F24781E77370043001A07245E5247245AF
:10117000EF20F0720100B2504561828041112AC611
:10118000B247FC473E854101828041112AC62EC4E8
:10119000B2472247F8C701004101828041112AC6A7
:1011A000B24783C707053E8541018280797106D623
:1011B0002AC62EC432C202CEB247BC4391EFB24718
:1011C0009C43D5E7B247DC433E85EF10903B2ACEE7
:1011D000B24723A2070061A8924785EFB24798471C
:1011E000B247BC433E86A2453A85EF20F079B2472C
:1011F0009847B247BC433E97B24798C7B247984713
:10120000B247DC436365F706B2479843B24798C7D5
:10121000B9A8B247D847B247BC433E86A2453A85F3
:10122000EF209076B247D847B247BC43B307F040AF
:101230003E97B247D8C7B247D847B2479C43637B73
:10124000F700B247D843B247BC43B307F0403E97DC
:10125000B247D8C712478947631BF700B2479C5F64
:1012600099C7B2479C5F1387F7FFB24798DFB24731
:101270009C5F13871700B24798DFF2473E85B25054
:1012800045618280011106CE2AC62EC4B247BC43F6
:101290009DCBB247D847B247BC433E97B247D8C769
:1012A000B247D847B247DC436366F700B24798437A
:1012B000B247D8C7B247D847B247BC433E86BA8583
:1012C0002245EF20706C0100F2400561828001111F
:1012D00006CE2AC6EF10D03625A0B247DC5395C7FC
:1012E000B247938747023E85EF10C025AA8799C36E
:1012F000EF104049B247BC471387F7FFB247B8C762
:10130000B247BC47E34BF0FC11A00100B2477D5748
:10131000B8C7EF10D035EF10B0321DA0B2479C4BCC
:101320008DC7B247C1073E85EF10C021AA8799C378
:10133000EF104045B247FC431387F7FFB247F8C3AD
:10134000B247FC43E34CF0FC11A00100B2477D57CB
:10135000F8C3EF10D0310100F2400561828079714D
:1013600006D62AC6EF10D02DB2479C5F81E785478D
:101370003ECE11A002CEEF10902FF2473E85B25024
:101380004561828001112AC6B24781E7737004303B
:1013900001A0B2479C5F81E785473ECE11A002CEF7
:1013A000F2473E8505618280797106D62AC6EF1024
:1013B0003029B247985FB247DC5F6315F700854775
:1013C0003ECE11A002CEEF10902AF2473E85B250D9
:1013D0004561828001112AC6B24781E773700430EB
:1013E00001A0B247985FB247DC5F6315F7008547FD
:1013F0003ECE11A002CEF2473E85056182800111EA
:101400002AC62EC402CE81A0178703001307872D9A
:10141000F2478E07BA979C4385E7178703001307A7
:10142000672CF2478E07BA97224798C317870300A5
:101430001307472BF2478E07BA973247D8C301A844
:10144000F24785073ECE72479D47E3FFE7FA01006A
:101450000561828001112AC602CE0DA817870300FC
:1014600013074728F2478E07BA97DC433247631CBD
:10147000F700178703001307E726F2478E07BA978E
:1014800023A0070001A8F24785073ECE72479D477B
:10149000E3F6E7FC010005618280797106D62AC671
:1014A0002EC432C2B2473ECEEF109019F247F84335
:1014B000FD576315F700F24723A20704F247B84728
:1014C000FD576315F700F24723A40704EF10301A05
:1014D000F2479C5F89EBF247938747021246A24589
:1014E0003E85EF00907E7245DD330100B2504561CC
:1014F0008280397106DE2ACE2ECC36C83AC63EC46A
:1015000042C246C0B287231BF100F24781E77370E5
:10151000043001A03247914763F5E700737004304F
:1015200001A08357610192453E85EF1080512AD476
:10153000A257638F0712A257985B83566101B707C2
:101540000040FD17B6978A07BA973ED29257F19B93
:101550003ED292578D8B81C77370043001A08357A0
:1015600061013E8782463246E2452255EF10E02770
:101570004246F2451255EFE09FF82A87A25798C3DA
:10158000A24781C7A247225798C3EF10700B97F765
:101590000100938727009C431387170097F70100EA
:1015A000938747FF98C397F701009387A7E49C436D
:1015B00095E397F701009387E7E3225798C397F7DE
:1015C0000100938727FD98438547631AF702EF10C0
:1015D000C02C35A097F70100938787FC9C4385E3D7
:1015E00097F70100938707E19C43DC573247636814
:1015F000F70097F701009387E7DF225798C397F723
:1016000001009387E7FA9C431387170097F70100BF
:10161000938707FA98C397F70100938767F9984370
:10162000A257B8C7A257D85797F70100938707F773
:101630009C4363F9E700A257D85797F701009387B7
:10164000E7F598C3A257D857BA878A07BA978A0787
:1016500017F701001307C7E63E97A2579107BE850B
:101660003A85EFE07FF485473ED6EF10500019A091
:10167000FD573ED6325785476313F70297F70100AF
:10168000938707F29C4381CF97F70100938787D612
:101690009C43DC57324763F4E700EFE03FD7B25793
:1016A0003E85F25021618280797106D62AC6EF10FC
:1016B0002079B24799E797F701009387A7D39C4316
:1016C00011A0B2473ECEF24791073E85EFE07FF88A
:1016D000F2479C5791C7F247E1073E85EFE07FF75D
:1016E000F2479107BE8517F501001305E5E7EFE026
:1016F000BFEB97F70100938767E89C4313871700B8
:1017000097F70100938787E798C397F701009387BE
:1017100027EA9C431387170097F70100938747E94F
:1017200098C3EF10C07497F70100938767E79C4355
:101730009DCB97F701009387E7CB9C437247631ECD
:10174000F70097F70100938727E79C4381C77370E1
:10175000043001A0EFE09FCB39A0EF10606EEF10D6
:10176000A04BEF10C0700100B250456182807971CA
:1017700006D62AC62EC402CEB24781E77370043063
:1017800001A0A24781E77370043001A097F7010020
:10179000938787E29C4381C77370043001A0A92D11
:1017A00097F70100938747DF9C433ECCB2479C43A9
:1017B0002247BA973ECAB2479C436247637EF7000E
:1017C000B2479C4352476374F7025247E24763F0C3
:1017D000E70285473ECE21A8B2479C435247636645
:1017E000F7005247E24763F4E70085473ECEB24731
:1017F000524798C3F24789CF97F70100938787BF75
:101800009C4391073E85EFE0DFE45245EF10001B5B
:1018100011252AC8C24799E3EFE05FBF0100B2502B
:1018200045618280797106D62AC602CEB247A9C325
:1018300097F70100938747D89C4381C773700430A2
:1018400001A05D2B97F70100938707D59C43324792
:10185000BA973ECC97F701009387C7B99C4391078D
:101860003E85EFE01FDF6245EF10401565232ACE6D
:10187000F24799E3EFE09FB90100B25045618280E1
:10188000797106D62AC6B2473ECCE24781E773702B
:10189000043001A097F701009387C7B59C436247C6
:1018A0006314F70002CEBDA0EF108059E247DC4B75
:1018B0003ECAEF10C05B97F70100938727C99C438E
:1018C0005247630AF70097F70100938767C89C4364
:1018D00052476315F70089473ECE2DA8524797F728
:1018E00001009387E7C9631BF700E2479C5781E734
:1018F0008D473ECE05A089473ECE29A8524797F78F
:101900000100938767C66315F70091473ECE19A083
:1019100085473ECEF2473E85B2504561828079715F
:1019200006D62AC6EF10C051B24799E797F70100D3
:10193000938747AC9C4311A0B2473ECEF247DC5799
:101940003ECCEF10C052E2473E85B25045618280E6
:10195000797106D62AC6EFE05FB9AA873ECEB247B4
:1019600099E797F701009387E7A89C4311A0B24736
:101970003ECCE247DC573ECAF2473E85EFE0FFB57A
:10198000D2473E85B25045618280797106D62AC61B
:101990002EC402CE2247914763F5E70073700430EE
:1019A00001A02247914763F4E70091473EC4EF103E
:1019B0002049B24799E797F701009387A7A39C4373
:1019C00011A0B2473ECCE247BC4B3ECA5247A247A9
:1019D000630AF70E2247D24763F6E70297F7010042
:1019E000938747A19C4362476308F70297F701007A
:1019F000938747A09C43DC572247636FF7008547D6
:101A00003ECE19A897F701009387C79E9C43624773
:101A10006314F70085473ECEE247DC573EC8E247F5
:101A2000B84BE247DC576315F700E2472247D8D7A7
:101A3000E2472247B8CBE2479C4F63C707001547F0
:101A4000A2471D8FE24798CFE247D44B4247BA875F
:101A50008A07BA978A0717F70100130767A6BA978C
:101A60006394F600854711A08147B9C7E247910703
:101A70003E85EFE01FBEE247D85797F701009387F6
:101A8000E7B19C4363F9E700E247D85797F70100B5
:101A90009387C7B098C3E247D857BA878A07BA97DF
:101AA0008A0717F701001307A7A13E97E24791079E
:101AB000BE853A85EFE05FAF724785476314F70054
:101AC000EFE0DF94EF10A03A0100B2504561828050
:101AD000797106D62AC6EF10A036B24799E797F774
:101AE0000100938727919C4311A0B2473ECEF24755
:101AF00091073E85EFE0FFB5F2479C5791C7F2474B
:101B0000E1073E85EFE0FFB4F2479107BE8517F588
:101B100001001305E5A6EFE03FA9EF10403597F768
:101B200001009387278D9C4372476319F70497F749
:101B300001009387E7A69C4389CF97F7010093871D
:101B4000A7A79C4381C77370043001A0EFE01F8CEE
:101B500091A097F701009387A7A2984397F70100F8
:101B6000938747A39C436319F70097F70100938776
:101B7000678823A0070039A8212729A897F7010023
:101B8000938707A29C4399C7EF10802BEF10C008E2
:101B9000EF10E02D0100B2504561828001112AC68C
:101BA00002CEB2473ECCB24781E77370043001A049
:101BB000E247D84B97F701009387879C6314F7009F
:101BC000854711A0814795C3E247985797F70100D1
:101BD00093874798630BF700E2479C5799E3854743
:101BE00011A0814799C385473ECEF2473E850561E6
:101BF0008280797106D62AC6B2473ECEB24781E7C7
:101C00007370043001A0F247C9C797E701009387BA
:101C1000677E9C437247630EF706EF1060227245A1
:101C2000B53F2A8785476314F706F24791073E853B
:101C3000EFE03FA2F247D85797F701009387079646
:101C40009C4363F9E700F247D85797F70100938761
:101C5000E79498C3F247D857BA878A07BA978A0792
:101C600017F701001307C7853E97F2479107BE8516
:101C70003A85EFE07F93F247D85797E701009387C3
:101C800067779C43DC576364F700EFE02FF8EF10B1
:101C9000001E0100B25045618280797106D62AC6C5
:101CA00002CEB2473ECCB24781E77370043001A048
:101CB000EFE0BF83AA873ECA6245CD352A878547B4
:101CC0006314F70897F701009387078F9C43A5E7F4
:101CD000E247D85797E701009387C7719C43DC57C9
:101CE0006364F70085473ECEE24791073E85EFE00B
:101CF0005F96E247D85797F701009387278A9C435E
:101D000063F9E700E247D85797F7010093870789FF
:101D100098C3E247D857BA878A07BA978A0717E75E
:101D200001001307E7793E97E2479107BE853A85A0
:101D3000EFE09F8711A8E247E107BE8517F5010094
:101D400013054581EFE05F86D2473E85EFE0EFF86F
:101D5000F2473E85B25045618280011106CE81482E
:101D600001488147014781461306004097E501007D
:101D70009385452917150000130585A5EFF06FF72A
:101D80002AC6324785476315F700EF10C06D2AC693
:101D9000324785476319F7027370043097F70100E3
:101DA000938747817D5798C397E701009387477FC3
:101DB000054798C397E701009387077E23A0070094
:101DC000EFE02FCE31A0B24781E77370043001A05D
:101DD0000100F24005618280411106C67370043033
:101DE00097E701009387C77B23A00700EFE0AFD9F7
:101DF0000100B2404101828097E701009387C77BD1
:101E00009C431387170097E701009387E77A98C3ED
:101E100001008280011106CE02C697E70100938778
:101E2000A7799C4381E77370043001A0EF10400153
:101E300097E70100938747789C431387F7FF97E75D
:101E400001009387677798C397E701009387C77668
:101E50009C436390071097E701009387A7739C4307
:101E60006389070E59A097E701009387A76EDC47A7
:101E7000DC473EC4A247E1073E85EFE08FFDA24765
:101E800091073E85EFE0EFFCA247D85797E70100A6
:101E90009387C7709C4363F9E700A247D85797E739
:101EA00001009387A76F98C3A247D857BA878A07BC
:101EB000BA978A0717E70100130787603E97A24782
:101EC0009107BE853A85EFE02FEEA247D85797E7F6
:101ED0000100938727529C43DC576368F70097E71C
:101EE00001009387676C054798C397E701009387C4
:101EF00067669C43ADFB97E701009387A76A9C4305
:101F00008DCF35A0452AAA8799C797E70100938707
:101F1000A769054798C397E701009387A7689C4383
:101F20001387F7FF97E701009387C76798C397E781
:101F30000100938727679C43F1F797E70100938798
:101F4000A766984385476316F70085473EC6EFE0CE
:101F5000EFCBEF00D071B2473E85F2400561828041
:101F6000011106CEEF00D06D97E701009387C7629D
:101F70009C433EC6EF00B06FB2473E85F24005611C
:101F80008280011106CEEFE04FD6AA873EC697E7C2
:101F90000100938767609C433EC4B2473E85EFE0F3
:101FA000CFD3A2473E85F2400561828097E70100CA
:101FB0009387475E9C433E858280797106D62AC608
:101FC0002EC432C202CE95473ECC3D3597E7010084
:101FD0009387475C9C4322476368F70CE247FD17F1
:101FE0003ECCF24796073247B306F7006247BA87FE
:101FF0008A07BA978A0717E701001307674CBA9751
:102000000546BE853685EF00902A2A87F247BA97A3
:102010003ECEE247E1F7F247960732473E9797E711
:1020200001009387A7529C430946BE853A85EF007D
:1020300010282A87F247BA973ECEF24796073247D2
:102040003E9797E701009387A7509C430946BE85BA
:102050003A85EF00D0252A87F247BA973ECEF2475D
:1020600096073247BA97114697E501009385C54F09
:102070003E85EF00D0232A87F247BA973ECEF2473B
:1020800096073247BA970D4697E501009385454F6D
:102090003E85EF00D0212A87F247BA973ECE92477D
:1020A00081C7924723A00700B533F2473E85B2505F
:1020B00045618280797106D602CE97E70100938749
:1020C000A74F9C436395071897E701009387C74C78
:1020D0009C431387170097E701009387E74B98C34A
:1020E00097E701009387474B9C433ECCE247B9EF0B
:1020F00097E70100938787459C439C4381C7737092
:10210000043001A097E70100938747449C433ECAEF
:1021100097E701009387C743984397E701009387A8
:10212000E74298C397E7010093878742524798C3D5
:1021300097E70100938787479C431387170097E72A
:1021400001009387A74698C3EF00102D97E7010081
:10215000938747469C4362476365F70C97E7010006
:102160009387C73E9C439C4399E3854711A08147D1
:1021700081CB97E701009387E7437D5798C355A02C
:1021800097E701009387873C9C43DC47DC473EC8C8
:10219000C247DC433EC66247B2476379F70097E720
:1021A000010093872741324798C3A5A8C2479107EA
:1021B0003E85EFE00FCAC2479C5791C7C247E1076F
:1021C0003E85EFE00FC9C247D85797E701009387D4
:1021D000E73C9C4363F9E700C247D85797E7010003
:1021E0009387C73B98C3C247D857BA878A07BA971D
:1021F0008A0717E701001307A72C3E97C2479107EC
:10220000BE853A85EFE04FBAC247D85797E701003D
:102210009387471E9C43DC57E362F7F485473ECE25
:1022200035BF97E701009387E71C9C43D85797E693
:1022300001009386E628BA878A07BA978A07B69775
:102240009843854763F1E70285473ECE29A897E783
:102250000100938727359C431387170097E70100F8
:102260009387473498C397E701009387E7339C43EC
:1022700099C385473ECEF2473E85B2504561828084
:10228000011106CE97E70100938707339C4381CB6A
:1022900097E7010093874731054798C339A297E72D
:1022A00001009387673023A0070097E70100938719
:1022B00067149C439C5B3EC6B7A7A5A59387575A56
:1022C0003EC4B2479C4322476314F702B2479107CA
:1022D0009C432247631EF700B247A1079C43224755
:1022E0006318F700B247B1079C4322476308F7041D
:1022F00097E7010093870710984397E701009387BA
:10230000670F9C4393874703BE853A85EF20100BE8
:1023100035A097E70100938767289C4381E7737096
:10232000043001A097E70100938747279C43138758
:10233000F7FF97E701009387672698C397E70100A7
:102340009387C725984397E6010093866617BA8757
:102350008A07BA978A07B6979C43C5DF97E70100BB
:102360009387C7239843BA878A07BA978A0717E7DC
:1023700001001307E714BA973EC29247DC43D843E3
:102380009247D8C39247D8439247A1076317F700F3
:102390009247DC43D8439247D8C39247DC43D8479F
:1023A00097E701009387070598C30100F240056194
:1023B0008280797106D62AC62EC4B24781E773702F
:1023C000043001A097E701009387C7029C43E1070F
:1023D000BE853245EFE04FA197E701009387870163
:1023E0009C4391073E85EFE0CFA62247FD5763103F
:1023F000F70297E701009387E7FF9C439107BE85AB
:1024000017E501001305C517EFE00F9A19A897E724
:102410000100938767189C432247BA973ECE7245C6
:10242000712B0100B25045618280797106D62AC6AF
:102430002EC432C2B24781E77370043001A097E71F
:102440000100938767179C4381E77370043001A0F4
:1024500097E70100938707FA9C43A246370700805D
:10246000558F98CF97E701009387C7F89C43E10702
:10247000BE853245EFE04F9397E70100938787F7DA
:102480009C4391073E85EFE0CF9C1247FD576310B8
:10249000F70297E701009387E7F59C439107BE8514
:1024A00017E501001305C50DEFE00F9019A897E798
:1024B00001009387670E9C431247BA973ECE724540
:1024C000F5290100B25045618280797106D62AC68D
:1024D0002EC432C2B24781E77370043001A097E77F
:1024E0000100938727F19C43E107BE853245EFE069
:1024F000AF8B97E701009387E7EF9C4391073E85F9
:10250000EFE02F95124785476310F70297E7010028
:10251000938747EE9C439107BE8517E5010013059D
:102520002506EFE06F8819A897E701009387C70693
:102530009C432247BA973ECE724549210100B250D2
:1025400045618280797106D62AC6B247DC47DC47EE
:102550003ECCE24781E77370043001A0E247E10717
:102560003E85EFE00F8F97E701009387E7049C43D8
:10257000A1EBE24791073E85EFE0AF8DE247D857E8
:1025800097E70100938787019C4363F9E700E247DF
:10259000D85797E701009387670098C3E247D85759
:1025A000BA878A07BA978A0717E70100130747F126
:1025B0003E97E2479107BE853A85EFD0FFFE11A80E
:1025C000E247E107BE8517E501001305A5F8EFD046
:1025D000BFFDE247D85797E701009387A7E19C43E7
:1025E000DC5763FBE70085473ECE97E70100938702
:1025F000A7FB054798C311A002CEF2473E85B25013
:1026000045618280797106D62AC62EC497E70100FB
:10261000938787FA9C4381E77370043001A02247B7
:10262000B70700805D8FB24798C3B247DC473ECC06
:10263000E24781E77370043001A03245EFE06F811B
:10264000E24791073E85EFE0CF80E247D85797E712
:1026500001009387A7F49C4363F9E700E247D8574A
:1026600097E70100938787F398C3E247D857BA8763
:102670008A07BA978A0717E70100130767E43E97AE
:10268000E2479107BE853A85EFD01FF2E247D8575F
:1026900097E70100938707D69C43DC5763FBE7006D
:1026A00085473ECE97E70100938707F0054798C31B
:1026B00011A002CEF2473E85B250456182804111A1
:1026C0002AC6B24781E77370043001A097E7010082
:1026D0009387C7ED9843B24798C397E70100938764
:1026E000A7EB9843B247D8C30100410182807971BA
:1026F00006D62AC62EC4B24781E77370043001A003
:10270000A24781E77370043001A01D2F97E70100F5
:10271000938787E89C433ECCA2479843FD576314B8
:10272000F70002CE91A8B247984397E7010093873C
:10273000E7E79C43630AF700B247DC4362476365FF
:10274000F70085473ECE0DA8B247DC4362471D8F98
:10275000A2479C436370F702A2479843B247D44311
:10276000E247B387F6403E97A24798C33245813F80
:1027700002CE19A085473ECEDD2DF2473E85B250F0
:102780004561828097E70100938707E2054798C378
:102790000100828001112AC6B24799C7B2473ECCD8
:1027A000E247FC473ECE11A002CEF2473E850561CE
:1027B000828001112AC62EC4B24791C7B2473ECECD
:1027C000F2472247F8C7010005618280011106CE59
:1027D0002AC6852297E70100938787CE98438547CD
:1027E000E3F9E7FEEFD09FC2EDB7397106DE2ACEDE
:1027F0002ECC32CA36C8BA872317F10002D625A0DC
:102800006247B257BA9703C70700F246B257B69766
:10281000238AE7026247B257BA9783C7070089CB7A
:10282000B25785073ED63257BD47E3FBE7FC11A000
:102830000100F247A38107045247914763F4E70080
:1028400091473ECAF2475247D8D7F2475247B8CBD2
:10285000F24723AA0704F24791073E85EFD0DFD362
:10286000F247E1073E85EFD03FD3F247724798CB5E
:102870001547D2471D8FF24798CFF2477247D8D3FA
:10288000F24723A20704F24723AC0704F24723AE22
:1028900007040100F25021618280011106CE02C6B8
:1028A0000DA03247BA878A07BA978A0717E701004F
:1028B000130707C1BA973E85EFD0DFCAB247850735
:1028C0003EC632479147E3FEE7FC17E501001305DA
:1028D00065C5EFD03FC917E501001305E5C5EFD089
:1028E0007FC817E501001305E5C6EFD0BFC717E5A0
:1028F0000100130565C7EFD0FFC617E501001305FA
:1029000025C8EFD03FC697E70100938727C417E794
:102910000100130727C198C397E70100938747C3B6
:1029200017E70100130747C198C30100F240056192
:102930008280011106CE8DA8EFF00FCC97E7010041
:10294000938787C29C4393B7170093F7F70F3EC650
:10295000EFF04FCCB247A9EBE52197E70100938751
:10296000A7C0DC47DC473EC4A24791073E85EFD0B5
:102970005FCE97E701009387E7C19C431387F7FF7A
:1029800097E70100938707C198C397E701009387F2
:10299000E7BE9C431387F7FF97E70100938707BEC5
:1029A00098C3F1212245912C97E70100938707BD39
:1029B0009C43D9F30100F24005618280011106CEEB
:1029C0002AC697E701009387E7A29C433247D8C302
:1029D00097E70100938747BC9C4332476372F70235
:1029E00097E701009387C7B6984397E7010093875D
:1029F00067A09C439107BE853A85EFD0FFBE35A8FE
:102A000097E70100938787B4984397E7010093877E
:102A1000679E9C439107BE853A85EFD0FFBC97E740
:102A20000100938727B99C4332476378F70097E703
:102A30000100938727B8324798C30100F24005612F
:102A40008280797106D6AA872EC42317F100A24787
:102A500089EB8357E1008A073E85EF104051AA8732
:102A600011A0A2473ECCE24785C313050006EF1034
:102A700000502ACEF24789C7F247624798DB31A05F
:102A80006245EF10C06111A002CEF24781CFF2473C
:102A9000985B8357E1008A073E869305500A3A8582
:102AA000EF104075F2473E85B25045618280397122
:102AB00006DE22DC2AC62EC432C202D6A2479C43BE
:102AC000638D070EA2473ED4A257DC43D843A257DA
:102AD000D8C3A257D843A257A1076317F700A2573C
:102AE000DC43D843A257D8C3A257DC43DC473ED2CD
:102AF000A2473ED08257DC43D8438257D8C382577F
:102B0000D8438257A1076317F7008257DC43D843A5
:102B10008257D8C38257DC43DC473ECEB257960774
:102B20003247BA97724798C3B25796073247BA9757
:102B3000724713074703D8C3B25796073247BA976D
:102B40007247384798C7B25796073247BA97124725
:102B5000D8C7B25796073247BA977247585798CB9B
:102B600012478D47631BF700F2479C5799C7B2572E
:102B700096073247BA970947D8C7B25796073247E0
:102B8000BA977247384BD8CBB25796073247BA97A5
:102B900023AC0700F247945BB257960732473304E1
:102BA000F70036850D20AA87231EF400B25785074B
:102BB0003ED672479257E31DF7F2B2573E85F25068
:102BC00062542161828001112AC602CE39A0B24727
:102BD00085073EC6F24785073ECEB24703C70700CA
:102BE0009307500AE305F7FEF24789833ECEF2478A
:102BF000C207C1833E8505618280011106CE2AC6C7
:102C0000B2479C5B3E85EF1080493245EF1020496A
:102C10000100F24005618280411197E7010093872E
:102C2000E7929C439C4399E3854711A0814781CB60
:102C300097E70100938707987D5798C305A097E70A
:102C400001009387A7909C43DC47DC473EC6B24710
:102C5000D84397E701009387E79598C301004101A6
:102C60008280411197D701009387C7789C433EC665
:102C7000B2473E8541018280411197E70100938769
:102C800027929C4381E785473EC619A897E7010034
:102C9000938787929C4381E789473EC611A002C66D
:102CA000B2473E8541018280797106D62AC6B24775
:102CB0003ECEB247F9C3F247D85797D70100938762
:102CC00067739C43DC57637AF70AF2479C4F63CCE7
:102CD000070097D701009387E7719C43DC5715479E
:102CE0001D8FF24798CFF247D44BF247D857BA8797
:102CF0008A07BA978A0717D701001307677CBA9724
:102D00006394F600854711A08147A5C3F247910758
:102D10003E85EFD01F9497D701009387A76D9C4302
:102D2000D857F247D8D7F247D85797E7010093878B
:102D3000E7869C4363F9E700F247D85797E701001D
:102D40009387C78598C3F247D857BA878A07BA9737
:102D50008A0717D701001307A7763E97F247910716
:102D6000BE853A85EFD05F8409A897D70100938785
:102D700067689C43D857F247D8D70100B2504561E5
:102D80008280797106D62AC6B2473ECC02CEB247BF
:102D9000DDC397D701009387E7659C4362476305CE
:102DA000F7007370043001A0E247FC4B81E77370B9
:102DB000043001A0E247FC4B1387F7FFE247F8CB52
:102DC000E247D857E247BC4B6307F706E247FC4BA4
:102DD000BDE3E24791073E85EFD0BF87E247B84B9E
:102DE000E247D8D7E247DC5715471D8FE24798CF17
:102DF000E247D85797D701009387477A9C4363F9F6
:102E0000E700E247D85797D701009387277998C3FF
:102E1000E247D857BA878A07BA978A0717D70100B7
:102E20001307076A3E97E2479107BE853A85EFD0C0
:102E3000AFF785473ECEF2473E85B250456182806E
:102E40007370043097D70100938787759C4391CFA7
:102E500097D701009387075A9C43F8430507F8C3A7
:102E600097D70100938707599C430100828097D729
:102E700001009387E7729C438DCB97D7010093871E
:102E800067579C43FC4395C397D7010093878756A8
:102E90009C43F8437D17F8C397D701009387875564
:102EA0009C43FC4399E3736004300100828041112C
:102EB00097D70100938707549C439C4F3EC697D7F2
:102EC0000100938727539C43D85797D701009387D6
:102ED00067529C4395463387E64098CFB2473E857C
:102EE0004101828097D701009387C7509C4389CBCB
:102EF00097D70100938707509C43F84B0507F8CB01
:102F000097D701009387074F9C433E858280797154
:102F100006D62AC62EC42D3797D701009387874D32
:102F20009C43BC4FADE397D701009387A74C9C43CC
:102F30000547F8CFA247A1CB97D701009387874BCE
:102F40009C4391073E85EFD0CFF02247FD57631099
:102F5000F70297D701009387E7499C439107BE8505
:102F600017D501001305C561EFD00FE419A897D755
:102F70000100938767629C432247BA973ECE724511
:102F8000353CEFD0AFC8E535653D97D70100938755
:102F900067469C43BC4F3ECCE2479DC3B24789CBBA
:102FA00097D70100938707459C4323AC070409A8E2
:102FB00097D70100938707449C43B84F7D17B8CF3C
:102FC00097D70100938707439C4323AE07044535F9
:102FD000E2473E85B25045618280797106D62AC6A5
:102FE0002EC432C236C0A93D97D7010093878740CF
:102FF0009C43F84F8947630DF70697D701009387E5
:10300000673F9C43B44F32471347F7FF758FB8CFE4
:1030100097D701009387073E9C430547F8CF824727
:10302000A1CB97D701009387E73C9C4391073E854E
:10303000EFD02FE20247FD576310F70297D7010048
:103040009387473B9C439107BE8517D50100130525
:103050002553EFD06FD519A897D701009387C75391
:103060009C430247BA973ECC6245893AEFD00FBAEB
:10307000FD3BF933924789CB97D701009387873778
:103080009C43B84F924798C397D7010093878736E0
:103090009C43F84F85476314F70002CE31A897D7B9
:1030A0000100938727359C43B44F22471347F7FF0E
:1030B000758FB8CF85473ECE97D70100938787336A
:1030C0009C4323AE07046533F2473E85B250456109
:1030D0008280797106D62AC62EC432C236C0854790
:1030E0003ECEB24781E77370043001A0B2473ECCB8
:1030F000813B824789C7E247B84F824798C3E2477E
:10310000FC4F3ECAE2470947F8CF1247914763EEAA
:10311000E70492471397270097D70100938707EF9B
:10312000BA97984397D70100938747EEBA9782875B
:10313000E247B84FA2475D8FE247B8CF3DA0E247D4
:10314000BC4F13871700E247B8CF05A0E2472247DC
:10315000B8CF21A8524789476306F700E2472247C4
:10316000B8CF21A002CE11A0010052478547631AB3
:10317000F706E24791073E85EFD0AFCDE247D8573B
:1031800097D70100938787419C4363F9E700E247A3
:10319000D85797D701009387674098C3E247D8571D
:1031A000BA878A07BA978A0717D7010013074731EA
:1031B0003E97E2479107BE853A85EFD0EFBEE247E2
:1031C0009C5781C77370043001A0E247D85797D746
:1031D0000100938727229C43DC5763F4E700EFD07C
:1031E000EFA27131F2473E85B2504561828039715C
:1031F00006DE2ACE2ECC32CA36C83AC685473ED61F
:10320000F24781E77370043001A0F2473ED4EFD05B
:10321000CFADAA873ED2C24789C7A257B84FC2478F
:1032200098C3A257FC4F3ED0A2570947F8CF524748
:10323000914763EEE704D2471397270097D7010021
:10324000938707DEBA97984397D70100938747DDA6
:10325000BA978287A257B84FE2475D8FA257B8CF7F
:103260003DA0A257BC4F13871700A257B8CF05A0A7
:10327000A2576247B8CF21A8025789476306F700D3
:10328000A2576247B8CF21A002D611A00100025771
:103290008547631DF708A2579C5781C77370043098
:1032A00001A097D70100938727319C43A1EBA25738
:1032B00091073E85EFD0EFB9A257D85797D70100B5
:1032C0009387C72D9C4363F9E700A257D85797D738
:1032D00001009387A72C98C3A257D857BA878A07AB
:1032E000BA978A0717D701001307871D3E97A25781
:1032F0009107BE853A85EFD02FAB11A8A257E10701
:10330000BE8517D501001305E524EFD0EFA9A2571C
:10331000D85797D701009387E70D9C43DC5763F795
:10332000E700B24781C7B247054798C392573E8529
:10333000EFD0AF9AB2573E85F25021618280797109
:1033400006D62AC62EC4B24781E77370043001A0A6
:10335000B2473ECEEFD06F99AA873ECCF247FC4FE2
:103360003ECAF2470947F8CFF247BC4F1387170010
:10337000F247B8CF52478547631DF708F2479C577D
:1033800081C77370043001A097D701009387C722CB
:103390009C43A1EBF24791073E85EFD08FABF247FC
:1033A000D85797D701009387671F9C4363F9E700BD
:1033B000F247D85797D701009387471E98C3F24723
:1033C000D857BA878A07BA978A0717D70100130711
:1033D000270F3E97F2479107BE853A85EFD0CF9CE5
:1033E00011A8F247E107BE8517D501001305851620
:1033F000EFD08F9BF247D85797D70100938787FF6D
:103400009C43DC5763F7E700A24781C7A247054703
:1034100098C3E2473E85EFD04F8C0100B250456122
:103420008280797106D62AC6B2473ECCE24799E738
:1034300097D70100938707FC9C4311A0E2473ECC3D
:103440000134E247F84F89476318F700E24723AE9B
:10345000070485473ECE11A002CE113CF2473E85BF
:10346000B25045618280011106CE02C61D2B97D74E
:1034700001009387A7179C439DC38148014881475A
:10348000094781461306004097D50100938585BA08
:10349000170500001305051BEFE0AF852AC6B247EC
:1034A00081E77370043001A0B2473E85F2400561A8
:1034B0008280397106DE2ACE2ECC32CA36C83AC690
:1034C000E24799E302D62DA81305C002EF00302A87
:1034D0002AD6B25795C7F121B257724798C3B2574F
:1034E000624798CFB2575247D8CFB257424798D386
:1034F000B2573247D8D3B25791073E85EFD0CF8924
:10350000E24781E77370043001A0B2573E85F25064
:1035100021618280397106DE2ACE2ECC32CA36C8AD
:103520003AC602D6F24781E77370043001A097D7FC
:1035300001009387A70B9C43B5CBE2473ED0D2470F
:103540003ED2F2473ED46247954763C4E704EFF0AA
:10355000AFF22A8789476310F70297D70100938754
:10356000E7089C43181081463246BA853E85EFD065
:103570002FBF2AD625A897D70100938727079C43FA
:10358000181081460146BA853E85EFD06FBD2AD618
:1035900031A897D70100938767059C43181081468F
:1035A0004246BA853E85EFD08FF22AD6B2573E8585
:1035B000F2502161828001112AC6B2473ECEB24745
:1035C00081E77370043001A0F2479C433E8505619A
:1035D0008280797106D62AC62EC497D701009387B8
:1035E00067009C43DC47DC473ECEF24791073E85AF
:1035F000EFD02F86F247D84F8547631BF702F2477B
:10360000984FB247BA97B2462246BE857245B92254
:103610002A878547631EF700014781463246814568
:103620007245CD3D2ACCE24781E77370043001A09A
:10363000F247DC53724582970100B25045618280A7
:10364000797106D62AC63C083E8541282ACEE24733
:10365000BE85724519206922FDB7797106D62AC642
:103660002EC4EFE06FF93C083E8545282ACEE2479C
:10367000B9EFA24799EB3247F24763E8E700EFE082
:103680006FF9F2453245B137A9A0A24781CF97D74C
:103690000100938767F59C439C4393B7170093F70A
:1036A000F70F3EC497D70100938747F494433247FE
:1036B000F247B307F7402246BE853685EFD0FFDDDF
:1036C000EFE04FF5AA8791E7EFC05FD419A0EFE0D4
:1036D0006FF40100B2504561828001112AC697D76C
:1036E0000100938727F09C439C4393B7170093F7FF
:1036F000F70F3E87B24798C3B2479C4391EB97D7E9
:103700000100938727EE9C43DC479C433ECE11A0EB
:1037100002CEF2473E8505618280797106D62AC6BF
:10372000EFE01F842ACE97D70100938767EC9C4374
:1037300072476377F700692AB247054798C321A00B
:10374000B24723A0070097D70100938767EA724723
:1037500098C3F2473E85B25045618280797106D6A2
:103760002AC62EC432C236C002CEB2472247D8C3C0
:10377000B247324798CB2247924763E8E7021247A5
:1037800082471D8FB2479C4F6365F70085473ECE49
:1037900099A097D70100938727E59843B2479107EF
:1037A000BE853A85EFC05FE43DA01247824763794A
:1037B000F700224782476365F70085473ECE21A880
:1037C00097D70100938707E29843B2479107BE85D8
:1037D0003A85EFC07FE1F2473E85B2504561828075
:1037E000797106D6D9A0A24763C0070CC2473ECE66
:1037F000F247DC4B91C7F24791073E85EFC07FE56A
:103800005C003E85193F2ACCA2472547636FF70825
:103810001397270097D7010093874782BA97984359
:1038200097D7010093878781BA9782873247F247FB
:103830009C4FBA973247BA866246BE857245393F79
:103840002A8785476313F706F247DC537245829750
:10385000F247D84F8547631AF7043247F2479C4F27
:10386000BA97014781463E868145724565312ACA2D
:10387000D24785EF7370043001A03247F24798CFEA
:10388000F2479C4F81E77370043001A0F247984FD4
:10389000E247BA97E2466246BE857245C13531A01D
:1038A0007245EF00C07F11A0010097D701009387F8
:1038B000E7D39C43380081460146BA853E85EFD068
:1038C0006FD8AA87E39107F20100B2504561828068
:1038D000797106D671A097D701009387A7D09C4332
:1038E000DC479C433ECC97D701009387A7CF9C43EE
:1038F000DC47DC473ECAD24791073E85EFC07FD503
:10390000D247DC5352458297D247D84F8547631937
:10391000F704D2479C4F6247BA973EC84247E247F6
:1039200063F4E702D2474247D8C3D247524798CB05
:1039300097D70100938707CB9843D2479107BE855D
:103940003A85EFC07FCA29A8014781466246814572
:103950005245C9362AC6B24781E77370043001A0C8
:1039600097D70100938707C89C439C43ADF797D72F
:103970000100938727C79C433ECE97D701009387CA
:10398000A7C6984397D701009387C7C598C397D711
:103990000100938767C5724798C30100B250456123
:1039A0008280411106C6EFF0AFC997D70100938717
:1039B000E7C39C43C9E717D50100130525C0EFC035
:1039C0007FBA17D501001305A5C0EFC0BFB997D7BF
:1039D0000100938727C117D70100130727BE98C39B
:1039E00097D70100938747C017D70100130747BE39
:1039F00098C30146B1451145EFC0FFD52A8797D737
:103A000001009387A7BE98C397D70100938707BE8D
:103A10009C4381E77370043001A097D7010093871E
:103A2000E7BC9C4389CF97D70100938727BC9C4371
:103A300097C50100938505633E85EFD05F9CEFF04D
:103A40000FC30100B24041018280797106D62AC6B7
:103A5000B2473ECEB24781E77370043001A0EFF069
:103A60002FBEF247DC4BB337F00093F7F70F3ECC95
:103A7000EFF0EFBFE2473E85B25045618280797139
:103A800006D62AC6B2473ECEB24781E773700430ED
:103A900001A0EFF0EFBAF2479C533ECCEFF02FBD00
:103AA000E2473E85B25045618280797106D62AC6CA
:103AB0002EC4B2473ECEB24781E77370043001A0F6
:103AC000EFF00FB8F247224798D3EFF04FBA01005A
:103AD000B25045618280011106CE714549292AC63E
:103AE000B24789CBB24723A00700B24791073E8572
:103AF000EFC05FA7B2473E85F24005618280397111
:103B000006DE2AC62EC432C236C0B2473ED402D226
:103B10001247B70700FFF98F81C77370043001A007
:103B2000924781E77370043001A0EFF0EF94AA8709
:103B300099E3824799E3854711A0814781E7737034
:103B4000043001A0EFE04FABA2579C433ED0A2450A
:103B5000324585240257A2475D8F9247F98F12475D
:103B60006310F7020257A247D98F3ED6A257984357
:103B7000924793C7F7FF7D8FA25798C302C025A035
:103B8000824799CFA257938647001247B70700058F
:103B9000D98F0246BE853685EFE03F8902D621A047
:103BA000A2579C433ED6EFE0EFA62ACE8247B1CB88
:103BB000F24799E3EFC09F85EFF06FAF2AD63257F7
:103BC000B7070002F98F85EBEFF08FA7A2579C4350
:103BD0003ED632579247F98F1247631AF700A25721
:103BE0009843924793C7F7FF7D8FA25798C3EFF092
:103BF0000FA885473ED23257B7070001FD17F98F4E
:103C00003ED6B2573E85F250216182805D7186C6F4
:103C10002ACE2ECC32CA36C83AC6F2473EDA02DC89
:103C200002D8F24781E77370043001A06247B707FA
:103C300000FFF98F81C77370043001A0E24781E76C
:103C40007370043001A0EFF02F83AA8799E3B24785
:103C500099E3854711A0814781E77370043001A083
:103C6000EFE08F99D2579C433ED64246E24532550B
:103C700075242AD4A25799CFB2573EDE02C6D24746
:103C8000A9CBD2579843E24793C7F7FF7D8FD2570E
:103C900098C381A0B24781E7B2573EDE1DA8D24744
:103CA00091C76257B7070001D98F3EDCC24791C761
:103CB0006257B7070004D98F3EDCD257938647007E
:103CC0006247E257D98F3246BE853685EFE0EFF581
:103CD00002DEEFE02F942AD2B247B9CB925799E394
:103CE000EFC0CFF2EFF0AF9C2ADE7257B7070002A9
:103CF000F98F8DEBEFF0CF94D2579C433EDE4246D6
:103D0000E2457255212CAA8799CBD24789CBD2574D
:103D10009843E24793C7F7FF7D8FD25798C3EFF0E0
:103D20000F9502D87257B7070001FD17F98F3EDED5
:103D3000F2573E85B64061618280797106D62AC607
:103D40002EC4B2473ECEB24781E77370043001A063
:103D50002247B70700FFF98F81C77370043001A0B5
:103D6000EFF00F8EF2479C433ECCF2479843A247B8
:103D700093C7F7FF7D8FF24798C3EFF04F8FE2476D
:103D80003E85B25045618280797106D62AC6B24717
:103D90003ECEEFC08FF5AA873ECCF2479C433ECA89
:103DA000E2473E85EFC06FF3D2473E85B250456192
:103DB00082805D7186C62AC62EC402DCB2473ED818
:103DC00002DAB24781E77370043001A02247B707D7
:103DD00000FFF98F81C77370043001A0C2579107AB
:103DE0003ED6B257A1073ED4EFE00F81B257DC4771
:103DF0003EDEC2579843A2475D8FC25798C3BDA805
:103E0000F257DC433ED2F2579C433ED002DA0257CF
:103E1000B70700FFF98F3ECE0257B7070001FD1725
:103E2000F98F3ED07247B7070004F98F89EBC2576C
:103E300098438257F98F89CF85473EDA11A8C25738
:103E400098438257F98F02576314F70085473EDA8B
:103E5000D2579DC37247B7070001F98F89C76257D0
:103E60008257D98F3EDCC2579843B7070002D98FDB
:103E7000BE857255EFE00FF992573EDE7257A2579A
:103E8000E310F7F8C2579843E25793C7F7FF7D8FC7
:103E9000C25798C3EFD01FF8C2579C433E85B64027
:103EA00061618280797106D62AC6B2473ECEF2475A
:103EB00091073ECCEFD05FF40DA0E247D847E24730
:103EC000A1076315F7007370043001A0E247DC47D7
:103ED000B70500023E85EFE0EFF2E2479C43F1FFB9
:103EE0007245752AEFD01FF30100B2504561828000
:103EF000011106CE2AC62EC4A24532455D3D010001
:103F0000F24005618280011106CE2AC62EC4A24568
:103F1000324525350100F2400561828001112AC633
:103F20002EC432C202CE924781EB3247A247F98FAC
:103F300081CF85473ECE09A83247A247F98F224755
:103F40006314F70085473ECEF2473E8505618280C7
:103F500001112AC6B2473ECCB24799E302CE21A056
:103F6000E2479C4F3ECEF2473E8505618280397123
:103F700006DE2AC602D2EFD03FE8975703009387A8
:103F800067689C4381EB55229757030093878767A7
:103F9000054798C3B24789CFA1473E87B247BA9732
:103FA0003EC6B2478D8B89C7B247F19B91073EC68B
:103FB000B247F9CB3247E567ED1763E7E70C975750
:103FC0000300938727633ED4975703009387876244
:103FD0009C433ED631A0B2573ED4B2579C433ED606
:103FE000B257DC43324763F5E700B2579C43E5F72D
:103FF000325797570300938767606307F708A25704
:104000009C432147BA973ED2B2579843A25798C3D0
:10401000B257D843B247B307F74021470607637842
:10402000F7043257B247BA973ECEB257D843B24799
:104030001D8FF247D8C3B2573247D8C3F247DC438B
:104040003ECC975703009387E75A3ED021A0825772
:104050009C433ED082579C43DC436247E3E9E7FE42
:1040600082579843F24798C38257724798C397C7BD
:104070000100938767399843B257DC431D8F97C778
:1040800001009387673898C3EFD0DFD8925799E340
:10409000EF00303292573E85F25021618280797173
:1040A00006D62AC6B2473ECCB247BDC3A147B30726
:1040B000F0406247BA973ECCE2473ECAEFD0DFD32A
:1040C000D247DC433EC8975703009387A7523ECEA2
:1040D00021A0F2479C433ECEF2479C43DC4342473B
:1040E000E3E9E7FEF2479843D24798C3F2475247C5
:1040F00098C3D247D84397C701009387E7309C43C2
:104100003E9797C701009387273098C3EFD09FD081
:104110000100B2504561828097C701009387C72E86
:104120009C433E85828001008280411197C7010037
:104130009387874CF19B3EC6975703009387874B25
:10414000324798C3975703009387C74A23A20700B3
:10415000975703009387874A65677117D8C39757A6
:1041600003009387A74923A00700B2473EC4A24794
:1041700065677117D8C3A24717570300130707488D
:1041800098C301004101828001112AC62EC432C2A7
:10419000A2473ECEB2473ECC3247A247D98F8D8B45
:1041A000A1E319A8F2479843E24798C3E247910771
:1041B0003ECCF24791073ECE9247F5173247BA9769
:1041C0006247E361F7FE29A87247930717003ECEC6
:1041D000E2479386170036CC034707002380E700A9
:1041E00032479247BA976247E360F7FEB2473E858F
:1041F0000561828001112AC62EC432C2324792471D
:10420000D98F8D8B9DEFA24793F7F70F3ECAD24708
:10421000A2075247D98F3ECAD247C2075247D98F09
:104220003ECAB2473ECE39A0F247138747003ACE86
:10423000524798C332479247BA977247E366F7FEF0
:104240001DA0B2473ECC11A8E247138717003ACC15
:1042500022471377F70F2380E70032479247BA9738
:104260006247E363F7FEB2473E8505618280011134
:104270002AC6B2473ECE21A0F24785073ECEF2477E
:1042800083C70700F5FB7247B247B307F7403E8587
:104290000561828001112AC62EC4B2471387170018
:1042A0003AC683C70700A30FF100A2471387170080
:1042B0003AC483C70700230FF1008347F10199C770
:1042C0000347F1018347E101E309F7FC0347F101EB
:1042D0008347E101B307F7403E8505618280011104
:1042E0002AC62EC4B2473ECE0100224793071700CC
:1042F0003EC4F2479386170036CE0347070023805B
:10430000E70083C70700F5F3B2473E850561828069
:1043100001112AC602CE02CC21A0B24785073EC6B3
:10432000B24703C7070093070002E308F7FEB2474E
:1043300003C707009307D0026309F700B24703C71A
:1043400007009307B0026311F704B24783C7070061
:10435000938737FD93B7170093F7F70F3ECCB2471B
:1043600085073EC615A07247BA878A07BA9786079F
:104370003ECEB247138717003AC683C7070093871C
:1043800007FD7247BA973ECEB24783C70700E1FFE9
:10439000E24789C7F247B307F04011A0F2473E85D4
:1043A0000561828001112AC69757030093878729E8
:1043B0009C4393861700175703001307A72814C3BD
:1043C00032471377F70F975603009386A62BB697BD
:1043D0002380E7003247A947630BF7009757030094
:1043E000938747269843930700046315F70497576C
:1043F0000300938727293ECE05A8F24713871700AD
:104400003ACE03C70700B70710F0938707F098C3A9
:1044100097570300938707239C431387F7FF97570A
:1044200003009387272298C3975703009387872118
:104430009C43E1F781473E85056182804D712326CB
:104440001114232481142322911423202115232EB7
:104450003113232C4113232A51132ACE2ECC32C8D8
:1044600036CA3AC63EC442C223260112B2473E8A29
:10447000814AC24752485286D6863E85C285EF1091
:10448000600DAA872E883E86C2868327C1121387B5
:1044900017002326E11232878A07141AB69723AE33
:1044A000E7EEB2473E848144D247268763E8E702BD
:1044B000D24726876396E700C247228763E0E70278
:1044C000B2473E8981494A86CE864245D245EF00B1
:1044D000B02AAA872E883EC842CA49BF010029A037
:1044E000F247E24512458297A2471387F7FF3AC485
:1044F0000327C112E346F7FE25A88327C1128A07C6
:10450000181ABA9703A7C7EF8327C1128A07141A8C
:10451000B69783A6C7EFA54763F5D7009307700545
:1045200019A093070003BA977247E2453E850297A8
:104530008327C1121387F7FF2326E112E34FF0FA16
:1045400001008320C114032481148324411403290E
:1045500001148329C113032A8113832A4113716132
:10456000828041112AC62EC4A2460547635ED70049
:10457000B2479C439D07E19B93868700324714C353
:1045800003A847009C4335A0224719CB3247184364
:1045900013064700B24690C21843BA87014811A8D3
:1045A0003247184313064700B24690C21843BA87F1
:1045B00001483E85C2854101828041112AC62EC430
:1045C000A2460547635ED700B2479C439D07E19B27
:1045D00093868700324714C303A847009C4305A86D
:1045E000224701CF3247184313064700B24690C214
:1045F0001843BA877D873A8819A8324718431306AB
:104600004700B24690C21843BA877D873A883E85F4
:10461000C28541018280397106DE22DC26DA2AC693
:104620002EC432C236C011A86307042492478507FE
:104630003EC2B247A24522858297924783C70700B0
:104640003E8493075002E311F4FE924785073EC271
:1046500092473EC893070002A30BF100FD573ECEE0
:10466000FD573ECC02D09247138717003AC283C74A
:1046700007003E849307D4FD130750056364F71EBB
:104680001397270097C701009387C79EBA9798434F
:1046900097C701009387079EBA9782879307D00236
:1046A000A30BF100C9B793070003A30BF10065BF8B
:1046B00002CC6247BA878A07BA978607A297938780
:1046C00007FD3ECC924783C707003E849307F00264
:1046D00063D687029307900363C2870292478507D8
:1046E0003EC2C1BF8247138747003AC09C433ECCBD
:1046F00039A0F247E3D907F602CEB5B70100F24779
:10470000E3D307F6E2473ECEFD573ECCA9BF825722
:1047100085073ED089BF8247138747003AC09C4334
:104720003247A2453E850297B1A2824713874700D0
:104730003AC0844389E497C4010093842493F247E8
:104740006357F004034771019307D0026301F70434
:10475000E247BE852685EF00E07F2A87F247998FE2
:104760003ECE11A8834771013247A2453E8502978C
:10477000F247FD173ECEF247E346F0FE09A8B247E6
:10478000A245228582978504F247FD173ECE83C756
:1047900004003E841DC0E247E3C307FEE247FD1765
:1047A0003ECCE247E3DD07FC09A8B247A24513056A
:1047B00000028297F247FD173ECEF247E347F0FE34
:1047C00055A88A8782553E85CD3BAA872E883ED440
:1047D00042D6A2573258C28763D90702B247A245D0
:1047E0001305D0028297A255325681470148B386FD
:1047F000B740368533B5A7003307C840B307A74095
:104800003E87B6873A883ED442D6A9473ED21DA8F5
:10481000A9473ED215A0A1473ED239A885473ED030
:10482000B247A245130500038297B247A24513057C
:1048300080078297C1473ED28A8782553E851533CD
:104840002AD42ED61257834771013E88F24722564A
:10485000B256A2453245DD3631A8B247A24522857F
:10486000829709A8B247A245130550028297C24712
:104870003EC20100D9B30100F2506254D25421610A
:10488000828041112AC6B70710F0938707F232479A
:1048900098C301A05D7106D62AC62EDA32DC36DE58
:1048A000BAC0BEC2C2C4C6C69C0891173ECEF2476B
:1048B000BE8632468145170500001305E5AEA13BD3
:1048C00081473E85B2506161828001112AC62EC4A3
:1048D0001EC2A2473ECEF2479C4332471377F70FE2
:1048E0002380E700F2479C4313871700F24798C3E1
:1048F0000100056182801D7106DE2AC62EC4B2C485
:10490000B6C6BAC8BECAC2CCC6CE9C103ED25C08DF
:104910004C0817060000130686FB7D779346F7FFC9
:104920000565130505803388A5003378E800136812
:10493000783B23A007013295698F13677733D8C37B
:1049400033F7D5009315470137870300130737392D
:104950004D8F98C73377D60093164701370703006A
:1049600013077706558FD8C70F100000B2473ED601
:104970009C10A1173ED422575C083E857C00BA8665
:104980002246BE854939B24723800700B2473E8799
:10499000B257B307F7403E85F2502561828041113E
:1049A000370510F0130545F408412AC6370510F005
:1049B000130505F408412AC4370510F0130545F422
:1049C0000841B248E39EA8FC32452A83814313176D
:1049D000030081462245AA850146B3E7B600336845
:1049E000C700370710F0130587F49305007D0146D3
:1049F000B386B700B688B3B8F8003307C800B387EA
:104A0000E8003E87B6873A881CC1232205010100D1
:104A100041018280411106C659379307000873A0EF
:104A200047300100B24041018280011106CE2AC602
:104A300017B5010013058579EFF0DFE50100F240BD
:104A400005618280011106CE2AC617B50100130543
:104A50006578EFF03FE40100F240056182807971F2
:104A600006D62AC602CE29A00100F24785073ECE0F
:104A70007247856793877738E3D8E7FE17B501005B
:104A80001305C575EFF01FE1F1BF411106C60945D9
:104A9000252A0100B24041018280011106CE02C6E2
:104AA000F92E2A878547630CF70017B50100130517
:104AB0006573EFF03FDEB24793E727003EC6B2478B
:104AC0003E85F24005618280011106CE02C6753F27
:104AD0001707000013076704814605469305400643
:104AE00017B501001305C571EFE0BF9C2AC6B24798
:104AF00099CBEFD0EFC6AA87014781463E86854510
:104B00003245EFE03FA102C4EFD02FA581473E859B
:104B1000F24005618280797106D62AC697C70100E6
:104B20009387878D9C431387470697C70100938718
:104B3000A78C98C397C701009387478C9C43138722
:104B4000470697C701009387678B98C397C70100F3
:104B50009387878A98438567938777BB63D5E704F4
:104B600097C70100938747899843FD7793878744C8
:104B70003E9797C701009387278898C3393F2ACE6D
:104B8000F24799EB97C70100938747879843896756
:104B90009387773263DBE700F2473E85EFF07FCE05
:104BA000EFD08FA321A0010011A00100B2504561F8
:104BB00082807370043001A00100828041112AC6F6
:104BC0002EC47370043001A05D7186C62AC6854765
:104BD0003EDE95473EDC9307803E3EDA02D8314503
:104BE000EFF0EFB82AD6014689457255EFB0BFB64F
:104BF0002A87B25798C3B2575257D8C3B2571757DC
:104C00000300130727AC98C73145EFF04FB62AD4FD
:104C1000B2579843A25798C3A2574257D8C3A25736
:104C200017570300130787AA98C78148014881478F
:104C30003247B2561306004097B501009385055DD3
:104C4000170500001305251CEFC0BF8A81480148E5
:104C500081470147A2561306004097B5010093858E
:104C6000655B1705000013054513EFC09F883145AC
:104C7000EFF0EFAF2AD2014689457255EFB0BFADD4
:104C80002A87925798C392574257D8C392571757BB
:104C900003001307C7A398C73145EFF04FAD2AD0E3
:104CA00092579843825798C382575257D8C3825716
:104CB00017570300130727A198C781480148814768
:104CC000014792561306004097B50100938505559C
:104CD0001705000013052513EFC0BF818148014867
:104CE0008147324782561306004097B501009385ED
:104CF0006553170500001305450AEFC08FFF3145C6
:104D0000EFF0EFA62ACE014689456255EFB0BFA469
:104D10002A87F24798C3F2475257D8C3F24717572A
:104D200003001307E79A98C73145EFF04FA42ACC48
:104D3000F2479843E24798C3E2475257D8C3E24745
:104D4000175703001307479898C7814801488147C0
:104D50000147F2461306004097B501009385054DC3
:104D60001705000013056503EFC0AFF8814801483F
:104D700081470147E2461306004097B5010093853D
:104D8000654B1705000013050508EFC08FF60100FD
:104D9000B64061618280797106D62AC6231B010064
:104DA000231F0100B2473ECCE2479843E247D0437D
:104DB000930761018146BE853A85EFB0DFD02A872F
:104DC00085476306F7008547231FF100F1BF83176E
:104DD000E10185E3E2479C4703D70700420741878B
:104DE00042074183050742074183420741872390D9
:104DF000E700835761018507C207C183231BF100C8
:104E000065B7797106D62AC6231F0100231E01004B
:104E1000B2473ECCE2479843E247D0439307610153
:104E20008146BE853A85EFB09FD72A878547E31331
:104E3000F7FE835761010357E101630AF7008357C7
:104E40006101231FF1008547231EF100E1B783179D
:104E5000C10185E3E2479C4703D70700420741872A
:104E60004207418305074207418342074187239058
:104E7000E7008357E1018507231FF10061BF41115E
:104E800085473EC602C475A81757030013078783DA
:104E9000A2478607BA9783D7070013970701418770
:104EA0009756030093860683A2478607B697839793
:104EB00007006313F70002C6175703001307878024
:104EC000A2478607BA9783D7070013970701418740
:104ED0009756030093860680A2478607B6972390CD
:104EE000E700174703001307677EA2478607BA97B4
:104EF00083D70700139707014187974603009386DE
:104F0000E67DA2478607B697839707006313F700ED
:104F100002C6174703001307677BA2478607BA97A5
:104F200083D70700139707014187974603009386AD
:104F3000E67AA2478607B6972390E700A24785073F
:104F40003EC422478947E3D1E7F4B2473E85410199
:104F500082800000B305B500930705006386B700A3
:104F600003C70700631607003385A740678000006A
:104F7000938717006FF09FFE130101FD232291021A
:104F8000232A5101232611022324810223202103F5
:104F9000232E3101232C4101232861012326710195
:104FA00023248101232291012320A101930A0500DA
:104FB00093840500639E06381304060093090500D8
:104FC00017B901001309892763F8C512B707010053
:104FD000138B05006378F6101307F00F3337C70003
:104FE00013173700B357E6003309F9008346090069
:104FF0003387E60093060002B386E640638C060022
:10500000B394D40033D7EA003314D600336B97003F
:10501000B399DA00935A040193850A0013050B0033
:10502000EF00902A1309050093850A00931B0401E1
:1050300013050B00EF00D02493DB0B019304050054
:105040009305050013850B00EF00D020131909010B
:1050500093D70901B367F900138A040063FEA70020
:10506000B3878700138AF4FF63E8870063F6A7001D
:10507000138AE4FFB3878700B384A74093850A00AF
:1050800013850400EF0050241309050093850A00DE
:1050900013850400EF00D01E9399090193040500C5
:1050A000930505001319090113850B0093D9090114
:1050B000EF00501AB36939011386040063FCA9009C
:1050C000B30934011386F4FF63E6890063F4A90091
:1050D0001386E4FF13140A013364C400130A0000AA
:1050E0006F000013B707000113070001E36CF6EE31
:1050F000130780016FF01FEF138A0600631A060082
:105100009305000013051000EF009017130405002D
:10511000B7070100637EF4129307F00F63F4870072
:10512000130A8000B35744013309F900034709000B
:105130009306000233074701B386E64063940612E4
:10514000B3848440130A1000135B040193050B0021
:1051500013850400EF0050171309050093050B0099
:1051600013850400931B0401EF00901193DB0B01E6
:10517000930405009305050013850B00EF00900DC7
:105180001319090193D70901B367F900938A040041
:1051900063FEA700B3878700938AF4FF63E8870064
:1051A00063F6A700938AE4FFB3878700B384A74020
:1051B00093050B0013850400EF001011130905007F
:1051C00093050B0013850400EF00900B93990901E0
:1051D00093040500930505001319090113850B00BD
:1051E00093D90901EF001007B36939011386040050
:1051F00063FCA900B30934011386F4FF63E6890058
:1052000063F4A9001386E4FF13940A013364C40015
:105210001305040093050A008320C10203248102C0
:1052200083244102032901028329C101032A810148
:10523000832A4101032B0101832BC100032C810030
:10524000832C4100032D010013010103678000003E
:10525000B7070001130A0001E366F4EC130A8001AA
:105260006FF05FEC3314D40033DAE400B399DA0062
:1052700033D7EA00935A0401B394D40093850A000B
:1052800013050A00336B9700EF00100413090500A3
:1052900093850A0013050A00931B0401EF00407E6A
:1052A00093DB0B01930405009305050013850B00A8
:1052B000EF00407A1319090113570B013367E90016
:1052C000138A0400637EA70033078700138AF4FF64
:1052D000636887006376A700138AE4FF33078700BB
:1052E000B304A74093850A0013850400EF00C07D36
:1052F0001309050093850A0013850400EF00407828
:10530000930405009305050013850B00EF008074DE
:1053100013170B011357070113190901B367E900AC
:105320001387040063FEA700B38787001387F4FF89
:1053300063E8870063F6A7001387E4FFB38787005D
:10534000131A0A01B384A740336AEA006FF0DFDF63
:1053500063ECD51EB707010063F4F6041307F00FE2
:10536000B335D7009395350033D7B60097B7010012
:105370009387C7ECB387E70003C70700130A00024F
:105380003307B700330AEA4063160A021304100019
:10539000E3E096E833B6CA00134416006FF05FE707
:1053A000B707000193050001E3E0F6FC93058001D7
:1053B0006FF09FFBB35CE600B3964601B3ECDC00F4
:1053C00033D4E40093DB0C01B397440133D7EA00F4
:1053D00093850B0013050400336BF700B3194601E6
:1053E000EF00806E1309050093850B001305040080
:1053F000139C0C01EF00C068135C0C0193040500C2
:105400009305050013050C00EF00C0641319090192
:1054100013570B013367E90013840400637EA70070
:10542000330797011384F4FF636897016376A7003D
:105430001384E4FF33079701B304A74093850B005F
:1054400013850400EF0040681309050093850B00E5
:1054500013850400EF00C062930405009305050066
:1054600013050C00EF00005F93170B0113190901DE
:1054700093D70701B367F9001386040063FEA70002
:10548000B38797011386F4FF63E8970163F6A700DB
:105490001386E4FFB387970113140401B70B0100CF
:1054A0003364C4001389FBFF337D240133F92901E0
:1054B000B384A7409305090013050D00EF00805940
:1054C000935C040193050900130B050013850C0080
:1054D000EF00405893D90901130C0500938509008A
:1054E00013850C00EF000057130905009385090090
:1054F00013050D00EF0000563305850193570B018E
:105500003385A70063748501330979019357050139
:10551000B387270163E6F402E392F4BCB707010006
:105520009387F7FF3375F50013150501337BFB00F7
:1055300033964A0133056501130A0000E37AA6CCCD
:105540001304F4FF6FF09FB9130A00001304000066
:105550006FF01FCC130101FB23248104232291044B
:10556000232E310323229103232611042320210516
:10557000232C4103232A510323286103232671038B
:10558000232481032320A103232EB101930C0500C2
:10559000938905001304050093840500639E062685
:1055A00013090600138A060097BA0100938A0AC9F4
:1055B00063F4C514B70701006376F6129307F00F82
:1055C00063F4C700130A8000B3574601B38AFA0098
:1055D00003C70A001305000233074701330AE540F9
:1055E000630C0A00B395490133D7EC003319460127
:1055F000B364B70033944C01935A090193850A00B0
:1056000013850400EF00404C9309050093850A00C0
:10561000131B090113850400EF008046135B0B0187
:105620009305050013050B00EF00C0429399090193
:1056300093570401B3E7F90063FAA700B387270182
:1056400063E6270163F4A700B3872701B384A7406B
:1056500093850A0013850400EF00004793090500B5
:1056600093850A0013850400EF00804113140401A0
:10567000930505009399090113050B0013540401C8
:10568000EF00403D33E48900637AA4003304240131
:10569000636624016374A400330424013304A4402A
:1056A00033554401930500008320C1040324810481
:1056B00083244104032901048329C103032A8103AC
:1056C000832A4103032B0103832BC102032C810294
:1056D000832C4102032D0102832DC1011301010519
:1056E00067800000B7070001130A0001E36EF6ECC3
:1056F000130A80016FF05FED631A06009305000046
:1057000013051000EF00C03713090500B7070100AB
:10571000637AF90E9307F00F63F42701130A8000F0
:10572000B3574901B38AFA0003C70A001305000200
:10573000B384294133074701330AE540E30E0AEAFF
:1057400033194901B3DAE900B395490133D7EC00C5
:1057500093540901336BB70013850A009385040045
:10576000EF0080369309050093850400931B09011F
:1057700013850A00EF00C03093DB0B019305050091
:1057800013850B00EF00002D9399090193570B012E
:10579000B3E7F90033944C0163FAA700B3872701FC
:1057A00063E6270163F4A700B3872701B38AA74004
:1057B0009385040013850A00EF000031930905006A
:1057C0009385040013850A00EF00802B93050500E4
:1057D00013850B00EF00002893150B019399090125
:1057E00093D50501B3E5B90063FAA500B38525019A
:1057F00063E6250163F4A500B3852501B384A540C4
:105800006FF09FDFB7070001130A0001E36AF9F0A8
:10581000130A80016FF0DFF0E3E8D5E8B707010075
:1058200063FCF604930BF00F33B5DB001315350062
:1058300033D7A60097B70100938747A0B387E70047
:1058400083CB070093050002B38BAB00338B75410C
:10585000631E0B0263E4360163EACC003384CC4060
:10586000B386D94033B58C00B384A6401305040039
:10587000938504006FF05FE3B70700011305000193
:10588000E3E8F6FA130580016FF09FFAB39666011C
:10589000335D7601336DDD0033D47901B395690151
:1058A00033DC7C0193540D01336CBC001305040000
:1058B00093850400B31A6601EF000021130A050066
:1058C000938504001305040033996C01931C0D01AA
:1058D000EF00001B93DC0C01130405009305050089
:1058E00013850C00EF000017131A0A0113570C015F
:1058F0003367EA00130A0400637EA7003307A70199
:10590000130AF4FF6368A7016376A700130AE4FF94
:105910003307A701B309A740938504001385090045
:10592000EF00801A93850400130405001385090015
:10593000EF000015930505009304050013850C0086
:10594000EF00401193150C011314040193D50501C8
:10595000B365B4001387040063FEA500B385A501F9
:105960001387F4FF63E8A50163F6A5001387E4FF3E
:10597000B385A501131A0A01B70C0100336AEA00C6
:105980001384FCFFB3778A0033F48A00B384A54004
:1059900013850700930504002326F100135A0A011A
:1059A000EF00400B930905009305040013050A005E
:1059B000EF00400A13DC0A01930D050093050C006B
:1059C00013050A00EF0000098327C100130A050030
:1059D00093050C0013850700EF00C0073305B501E0
:1059E00013D709013307A7006374B701330A9A017B
:1059F000B70701009387F7FF935507013377F70047
:105A000013170701B3F7F900B3854501B307F70092
:105A100063E6B400639EB400637CF90033865741AB
:105A2000B3B7C700B385A541B385F540930706001A
:105A3000B307F9403339F900B385B440B385254144
:105A400033947501B3D767013365F400B3D56501AD
:105A50006FF09FC5130605001305000093F61500AF
:105A6000638406003305C50093D515001316160090
:105A7000E39605FE678000006340050663C60506E1
:105A800013860500930505001305F0FF630C06025D
:105A900093061000637AB6006358C0001316160010
:105AA00093961600E36AB6FE1305000063E6C50090
:105AB000B385C5403365D50093D61600135616003E
:105AC000E39606FE6780000093820000EFF05FFB24
:105AD00013850500678002003305A04063D80500E8
:105AE000B305B0406FF0DFF9B305B040938200001A
:105AF000EFF01FF93305A040678002009382000099
:105B000063CA0500634C0500EFF09FF7138505009D
:105B100067800200B305B040E35805FE3305A0409E
:0C5B2000EFF01FF63305B0406780020074
:02000004800278
:1000000049444C45000000006031FEFF2831FEFFEE
:100010003631FEFF4431FEFF4C31FEFF7032FEFFF1
:100020003832FEFF4632FEFF5432FEFF5C32FEFFE6
:10003000546D722053766300F437FEFFF437FEFFF1
:10004000F437FEFF7238FEFF4238FEFF6838FEFFCD
:10005000F437FEFFF437FEFF7238FEFF4238FEFF32
:10006000546D725100000000286E756C6C29000000
:10007000F645FEFFF447FEFFEA47FEFFF447FEFFAA
:10008000F447FEFFF447FEFFF447FEFF7446FEFF11
:10009000F447FEFFF447FEFF2C46FEFF8246FEFFBC
:1000A000F447FEFF3646FEFF4046FEFF4046FEFF99
:1000B0004046FEFF4046FEFF4046FEFF4046FEFF34
:1000C0004046FEFF4046FEFF4046FEFFF447FEFF6F
:1000D000F447FEFFF447FEFFF447FEFFF447FEFF40
:1000E000F447FEFFF447FEFFF447FEFFF447FEFF30
:1000F000F447FEFFF447FEFFF447FEFFF447FEFF20
:10010000F447FEFFF447FEFFF447FEFFF447FEFF0F
:10011000F447FEFFF447FEFFF447FEFFF447FEFFFF
:10012000F447FEFFF447FEFFF447FEFFF447FEFFEF
:10013000F447FEFFF447FEFFF447FEFFF447FEFFDF
:10014000F447FEFFF447FEFFF447FEFFF447FEFFCF
:10015000F447FEFFF447FEFFF447FEFFF447FEFFBF
:10016000F447FEFFF447FEFFF447FEFFF447FEFFAF
:10017000A646FEFF5247FEFFF447FEFFF447FEFF90
:10018000F447FEFFF447FEFFF447FEFFF447FEFF8F
:10019000F447FEFF9E46FEFFF447FEFFF447FEFFD6
:1001A000A647FEFFAC47FEFFF447FEFFF447FEFF05
:1001B000BA46FEFFF447FEFFA047FEFFF447FEFFEE
:1001C000F447FEFFC447FEFF6D69616F750A0000CA
:1001D0006D69616F75320A0068756E6772790A0021
:1001E0004572726F7220696E20416C74426C636B51
:1001F00051207461736B73200D0A000043686563BE
:100200006B54696D6572000051436F6E734231002B
:100210005150726F644232005150726F6442330029
:1002200051436F6E734234005150726F6442350017
:1002300051436F6E73423600000102020303030351
:100240000404040404040404050505050505050566
:100250000505050505050505060606060606060646
:10026000060606060606060606060606060606062E
:100270000606060606060606070707070707070716
:1002800007070707070707070707070707070707FE
:1002900007070707070707070707070707070707EE
:1002A00007070707070707070707070707070707DE
:1002B00007070707070707070808080808080808C6
:1002C00008080808080808080808080808080808AE
:1002D000080808080808080808080808080808089E
:1002E000080808080808080808080808080808088E
:1002F000080808080808080808080808080808087E
:10030000080808080808080808080808080808086D
:10031000080808080808080808080808080808085D
:10032000080808080808080808080808080808084D
:08033000080808080808080885
:100338001000000000000000017A5200017C010159
:100348001B0D02004C00000018000000244CFEFFAA
:10035800DC05000000440E30708903950781018890
:100368000292049305940696089709980A990B9A9D
:100378000C0370020AC144C844C944D244D344D4CB
:1003880044D544D644D744D844D944DA440E00442A
:100398000B0000005000000068000000B051FEFF94
:1003A8000005000000440E507488028903930599E3
:1003B8000B810192049406950796089709980A9A62
:1003C8000C9B0D0320010AC144C844C944D244D33C
:1003D80044D444D544D644D744D844D944DA44DB39
:0803E800440E00440B0000006C
:1003FC00AAAAAAAA08000000FC8F010004000000B1
:040000058000004037
:00000001FF
